:0600000000308A00102808
:10000800FF000308F9000408FA000A08FB007E084C
:10001800FC000A128A11A9293D3084000130FE0033
:100028005B30FF0021208000840A0408703A03191D
:100038002528FF0A0319FE0A16287E088A007F0869
:1000480082000A128A1128280A128A118E210A129D
:100058008A11031083160317003003180130880033
:100068000130831203138500FF308600FF308700BC
:100078000030F2000030F3000030F6000030F700E6
:100088000530F4000030F5007708803AF800803039
:100098007802031D51280830760203185428552881
:1000A80066280130F8007608073C013E5D280310F9
:1000B800F80DFF3E031D5B287808FF3A8600FF30E5
:1000C80087007628FF3086000130F80076080F3C5C
:1000D800013E70280310F80DFF3E031D6E287808B6
:1000E800FF3A8700031472086D3E84008313760874
:1000F80000078400000D85007408F001F0077508FA
:10010800F101F1077108803AF80080307802031D88
:100118008F28013070020318922893289428A72862
:10012800FF30F0070318F10AFF30F1077108803A31
:10013800F80080307802031DA328013070020318EC
:10014800A628A7289428013085000518AC28AD28D2
:1001580040290C3076067704031DB328B428D32829
:10016800013085000130F2070318F30A0030F30765
:100178007308803AF80080307802031DC5280330E0
:100188007202031CC828C928CD280030F2000030AC
:10019800F300CE28051CD128D228CE2840290D30BE
:1001A80076067704031DD928DA28F7280130F407E2
:1001B8000318F50A0030F5077508803AF800803012
:1001C8007802031DE9280B307402031CEC28ED2883
:1001D800F1280A30F4000030F500F228051CF52853
:1001E800F628F22840290E3076067704031DFD28EC
:1001F800FE281B29FF30F4070318F50AFF30F5071E
:100208007508803AF80080307802031D0D29023005
:10021800740203181029112915290230F40000303E
:10022800F5001629051C19291A29162940290F3005
:1002380076067704031D21292229402901308500EB
:10024800F7308700831603130D15831203130B175A
:10025800831603138E16831203138B136300000097
:10026800831603138E12831203130D118B173C2967
:10027800051C3F2940293C290130F6070318F70AD5
:100288000030F7077708803AF80080307802031DBD
:100298004F2910307602031C522953295729003060
:1002A800F6000030F70048280A128A1110281F3477
:1002B8001F341F341F341F341F341F341F341F349E
:1002C8001F341F341F341F341F341F341F341F348E
:1002D800143416340934003400340A34153416340E
:1002E8000934003400341F34113411340E341F34EF
:1002F80004340A341134003406340B340D34003419
:10030800063409340F3400340F34083407344D34BC
:100318005D343D3403100030031801308B00803009
:10032800831603138100031000300318013087007F
:1003380040308F0001308500031000300318013071
:100348008600831203138B1708007C08FE007B08C5
:100358008A007A08840079088300FF0E7F0E09005E
:04400E00F52CFF3E50
:00000001FF
